:10000000C2C00000DEC00000DCC00000E3C1000090
:10001000D8C00000D6C00000D4C00000D2C000008C
:10002000D0C0000030C20000CCC00000CAC0000038
:10003000C8C00000C6C00000C4C00000C2C00000AC
:10004000C0C00000BEC00000BCC00000BAC00000BC
:10005000B8C00000B6C00000B4C00000B2C00000CC
:10006000B0C00000AEC00000ACC00000AAC00000DC
:10007000A8C00000A6C00000A4C00000A2C00000EC
:10008000A0C000009EC000009CC0000000407A108C
:10009000F35A00A0724E18090010A5D4E80000E839
:1000A0007648170000E40B54020000CA9A3B000097
:1000B00000E1F505000080969800000040420F0026
:1000C0000000A08601000000102700000000E803E7
:1000D000000000006400000000000A0000000000B2
:1000E0000100000000002C76D888DC674F0823DF71
:1000F000C1DFAE59E1B1B796E5E3E453C63AE65144
:10010000997696E8E6C28426EB898C9B62ED407C6A
:100110006FFCEFBC9C9F40F2BAA56FA5F490055A06
:100120002AF75C936B6CF9676DC11BFCE0E40D472B
:10013000FEF520E6B500D0ED902E0300943577054E
:100140000080841E080000204E0A000000C80C3306
:100150003333330F986E12831141EF8D2114893B95
:10016000E65516CFFEE6DB18D1844B381BF77C1D15
:10017000901DA4BBE424203284725E228100C9F168
:1001800024ECA1E53D2711241FBECFEFD0E1DEBF57
:10019000CDBF11E0A0E0B1E0E6EBF3E100E00BBF82
:1001A00002C007900D92A832B107D9F721E0A8E26A
:1001B000B1E001C01D92A433B207E1F732D10C9433
:1001C000D9091ECF9BB321E030E002C0220F331FBC
:1001D0008A95E2F7292B2BBB08959BB321E030E0F1
:1001E00002C0220F331F8A95E2F7209529232BBBEB
:1001F000089586E090E0E6DF83EC99E00197F1F75F
:1002000000C0000086E090E0E8DF87E893E1019716
:10021000F1F700C000000895CF93C82F85BB84E09C
:1002200090E0D0DFE6DFC295C07FC5BB84E090E000
:10023000C9DFDFDFCF910895CF93C82F85BB84E05E
:1002400090E0CBDFD6DFC295C07FC5BB84E090E0F5
:10025000C4DFCFDFCF91089581E0EEDF87E893E13F
:100260000197F1F700C0000080E8E6CF0895CF9332
:100270008FEF84BB85BB8ABB15BA1BBAC0E2C5BB76
:10028000B8DFC5BBB6DF80E885BBB3DF15BAB1DF29
:1002900080EF85BBAEDF15BAACDF80E685BBA9DF9A
:1002A00082E0CADFA6DFCF910895CF93DF93EC0100
:1002B00002C0B2DF219688818111FBCFDF91CF91FF
:1002C00008954F925F926F927F92AF92BF92CF92BA
:1002D000DF92EF92FF920F931F93CF93DF9300D0A3
:1002E00000D000D0CDB7DEB7CDB6DEB620E030E02E
:1002F0004AE754E4AFD12B013C0183E291E09F93A4
:100300008F931F921F921F921F921CD37C019E01FC
:100310002F5F3F4F5901890122E042E0C301B20142
:10032000F2D2C70101960F900F900F900F900F908F
:100330000F902DB73EB7281B390B0FB6F8943EBF70
:100340000FBE2DBF0DB71EB70F5F1F4F37E0E30E77
:10035000F11CBF92AF9281E291E09F938F93FF9245
:10036000EF921F930F93EED2802F912F9EDF8DB7C8
:100370009EB708960FB6F8949EBF0FBE8DBF0FB6FE
:10038000F894DEBE0FBECDBE26960FB6F894DEBF43
:100390000FBECDBFDF91CF911F910F91FF90EF90D6
:1003A000DF90CF90BF90AF907F906F905F904F9015
:1003B000089520910001222351F00197439738F4CA
:1003C000D1D01092000161E080E092E0BEC00895BB
:1003D00004C108951F920F920FB60F9211240BB60D
:1003E0000F922F933F934F935F936F937F938F93CE
:1003F0009F93AF93BF93EF93FF93FCD0FF91EF9147
:10040000BF91AF919F918F917F916F915F914F912C
:100410003F912F910F900BBE0F900FBE0F901F902A
:100420001895CCD024DFA0D088EE91E027D089EDBC
:1004300091E0FED087EA91E60197F1F700C0000055
:100440000BDF60E088E592E080D006DFF6D039DF90
:1004500084E690E0A4D0F9CF90912F01911107C0CC
:10046000E82FF0E0EF5FFE4F808183B90895E82F19
:10047000F0E0E75FFE4F808183B9089590933101EA
:100480008093300108951F920F920FB60F9211249E
:100490000BB60F922F933F934F935F936F937F937E
:1004A0008F939F93AF93BF93EF93FF9314BC80916F
:1004B0002801D2DF80912801873020F48F5F80935C
:1004C000280130C0109228018091290190912A01C1
:1004D000009799F480912F01811104C081E08093ED
:1004E0002F0102C010922F0180912B0190912C01BD
:1004F00090932A018093290115C09C012F71332705
:10050000232B39F4E0913001F0913101309709F05B
:1005100009958091290190912A01019790932A01D0
:1005200080932901FF91EF91BF91AF919F918F919E
:100530007F916F915F914F913F912F910F900BBEE3
:100540000F900FBE0F901F90189590932A018093E3
:10055000290190932C0180932B0160932F018CE053
:1005600085BD089515BC08958FEF82B9809364000E
:1005700081E08093650013B887E383BD80E887BF7F
:100580007894089520E030E006C043E04A95F1F702
:1005900000002F5F3F4F28173907B8F3089520E078
:1005A00030E008C0E3ECF9E03197F1F700C000005B
:1005B0002F5F3F4F28173907A8F308958FEF8093D7
:1005C000640011BA80E380936A0089B7846089BFB0
:1005D0001FBC8CE08EBD78940895CF93DF93C5E661
:1005E000D0E018828AE090E0CDDF81E08883DF915F
:1005F000CF91089580911101813041F480E2809380
:100600006A001DBC1CBC10921101089580E3809308
:100610006A008CB59DB590932E0180932D01E091D9
:100620003201F0913301099581E080931101089521
:100630009093330180933201089560912D01709160
:100640002E0180E090E06ED020E030E04AE253E4FA
:10065000F7C008950CD0BAC0B2D040F0A9D030F0A5
:1006600021F45F3F19F09BC05111E4C09EC0BFD080
:1006700098F39923C9F35523B1F3951B550BBB2769
:10068000AA2762177307840738F09F5F5F4F220F16
:10069000331F441FAA1FA9F333D00E2E3AF0E0E80F
:1006A00030D091505040E695001CCAF729D0FE2F5B
:1006B00027D0660F771F881FBB1F261737074807ED
:1006C000AB07B0E809F0BB0B802DBF01FF279358A3
:1006D0005F4F2AF09E3F510568F061C0ABC05F3F9D
:1006E000ECF3983EDCF3869577956795B795F7958B
:1006F0009F5FC9F7880F911D9695879597F9089583
:10070000E1E0660F771F881FBB1F6217730784071E
:10071000BA0720F0621B730B840BBA0BEE1F88F72D
:10072000E0950895E89409C097FB3EF49095809574
:10073000709561957F4F8F4F9F4F9923A9F0F92FA7
:1007400096E9BB279395F695879577956795B79525
:10075000F111F8CFFAF4BB0F11F460FF1BC06F5F0B
:100760007F4F8F4F9F4F16C0882311F096E911C01D
:10077000772321F09EE8872F762F05C0662371F03E
:1007800096E8862F70E060E02AF09A95660F771F52
:10079000881FDAF7880F9695879597F9089597F946
:1007A0009F6780E870E060E008959FEF80EC089517
:1007B00000240A9416161706180609060895002440
:1007C0000A9412161306140605060895092E0394BA
:1007D000000C11F4882352F0BB0F40F4BF2B11F42E
:1007E00060FF04C06F5F7F4F8F4F9F4F089557FD8D
:1007F0009058440F551F59F05F3F71F04795880F8F
:1008000097FB991F61F09F3F79F087950895121625
:1008100013061406551FF2CF4695F1DF08C01616D1
:1008200017061806991FF1CF869571056105089482
:100830000895E894BB2766277727CB0197F9089599
:100840000BD0C4CFB5DF28F0BADF18F0952309F03C
:10085000A6CFABCF1124EECFCADFA0F3959FD1F383
:10086000950F50E0551F629FF001729FBB27F00D5E
:10087000B11D639FAA27F00DB11DAA1F649F6627B3
:10088000B00DA11D661F829F2227B00DA11D621F02
:10089000739FB00DA11D621F839FA00D611D221FBC
:1008A000749F3327A00D611D231F849F600D211DA0
:1008B000822F762F6A2F11249F5750408AF0E1F043
:1008C00088234AF0EE0FFF1FBB1F661F771F881F8C
:1008D00091505040A9F79E3F510570F060CFAACFCC
:1008E0005F3FECF3983EDCF3869577956795B79577
:1008F000F795E7959F5FC1F7FE2B880F911D9695A1
:10090000879597F90895EF920F931F93CF93DF93F5
:10091000E80147FD02C034E001C034E1042E000CC0
:10092000550B57FF03C0519541955109E32E022FF6
:10093000242FAE0140D2CE01DF91CF911F910F91B4
:10094000EF9008950F931F93CF93DF93CDB7DEB74A
:100950002E970FB6F894DEBF0FBECDBF0D891E894E
:100960008F89988D26E02C831A83098397FF02C014
:1009700080E090E801979E838D83AE01455E5F4FD6
:10098000698D7A8DCE01019619D04D815E8157FD1A
:100990000AC02F813885421753070CF49A01F801D9
:1009A000E20FF31F10822E960FB6F894DEBF0FBE33
:1009B000CDBFDF91CF911F910F9108952F923F925C
:1009C0004F925F926F927F928F929F92AF92BF925F
:1009D000CF92DF92EF92FF920F931F93CF93DF930B
:1009E000CDB7DEB72B970FB6F894DEBF0FBECDBFE5
:1009F0006C017B018A01FC0117821682838181FFD1
:100A0000BFC1CE0101963C01F6019381F70193FD30
:100A1000859193FF81917F01882309F4ADC18532CF
:100A200039F493FD859193FF81917F01853221F403
:100A3000B60190E024D4E8CF912C212C312CFFE199
:100A4000F315D8F08B3279F038F4803279F08332B4
:100A5000A1F4232D20611DC08D3261F0803369F433
:100A6000232D216016C0832D8260382EE32DE46093
:100A70003E2E2AC0F32DF8601DC037FC2DC020ED9E
:100A8000280F2A3040F08E32B9F436FC75C1232D80
:100A90002064322E19C036FE06C08AE0989E200DD2
:100AA0001124922E11C0EAE02E9E200D1124222E38
:100AB000F32DF0623F2E08C08C3621F4832D806820
:100AC000382E02C0883641F4F70193FD859193FFDB
:100AD00081917F018111B3CF982F9F7D95549330E1
:100AE00028F40C5F1F4F9FE399830DC0833631F0CC
:100AF000833771F0833509F055C020C0F80180813B
:100B000089830E5F1F4F88248394912C530112C058
:100B10002801F2E04F0E511CF801A080B18036FE92
:100B200003C0692D70E002C06FEF7FEFC5019CD359
:100B30004C018201F32DFF773F2E15C0280122E0E2
:100B4000420E511CF801A080B18036FE03C0692D11
:100B500070E002C06FEF7FEFC5017BD34C01F32D36
:100B6000F0683F2E820133FC19C0822D90E0881678
:100B70009906A0F4B60180E290E081D32A94F5CFE3
:100B8000F50137FC859137FE81915F01B60190E058
:100B900076D321102A9421E0821A910881149104BD
:100BA00079F7E1C0843611F0893639F5F80137FE5E
:100BB00007C060817181828193810C5F1F4F08C0E3
:100BC00060817181072E000C880B990B0E5F1F4FFF
:100BD000F32DFF763F2E97FF09C090958095709575
:100BE00061957F4F8F4F9F4FF0683F2E2AE030E096
:100BF000A30181D3882E861844C0853731F4232D74
:100C00002F7EB22E2AE030E025C0932D997FB92E99
:100C10008F36C1F018F4883579F0AEC0803719F0FE
:100C2000883721F0A9C0E92FE061BE2EB4FE0DC0C7
:100C3000FB2DF460BF2E09C034FE0AC0292F2660A8
:100C4000B22E06C028E030E005C020E130E002C04E
:100C500020E132E0F801B7FE07C060817181828136
:100C600093810C5F1F4F06C06081718180E090E02E
:100C70000E5F1F4FA3013FD3882E8618FB2DFF77F1
:100C80003F2E36FE0DC0232D2E7FA22E891458F440
:100C900034FE0BC032FC09C0832D8E7EA82E05C009
:100CA000B82CA32C03C0B82C01C0B92CA4FE0FC0D3
:100CB000FE01E80DF11D8081803321F49A2D997E8B
:100CC000A92E09C0A2FE06C0B394B39404C08A2D15
:100CD000867809F0B394A3FC10C0A0FE06C0B2143D
:100CE00080F4280C922C9B180DC0B21458F4B60155
:100CF00080E290E0C4D2B394F8CFB21418F42B1869
:100D000002C0982C212CA4FE0FC0B60180E390E015
:100D1000B6D2A2FE16C0A1FC03C088E790E002C0D4
:100D200088E590E0B6010CC08A2D867851F0A1FECE
:100D300002C08BE201C080E2A7FC8DE2B60190E028
:100D40009ED2891430F4B60180E390E098D29A9450
:100D5000F8CF8A94F301E80DF11D8081B60190E08F
:100D60008ED28110F6CF222009F44ECEB60180E259
:100D700090E085D22A94F7CFF6018681978102C050
:100D80008FEF9FEF2B960FB6F894DEBF0FBECDBF4F
:100D9000DF91CF911F910F91FF90EF90DF90CF9057
:100DA000BF90AF909F908F907F906F905F904F908B
:100DB0003F902F9008958F929F92AF92BF92CF92C3
:100DC000DF92EF92FF920F931F93CF93DF93CDB7F4
:100DD000DEB729970FB6F894DEBF0FBECDBF6A010C
:100DE000122FB02E2BE3201720F0FF24F394F00EE7
:100DF00002C02CE3F22E0F2D27E0AE014F5F5F4FB4
:100E000050D1BC014981842F8970813031F0E1FCDF
:100E100006C0E0FE06C090E205C09DE203C09BE272
:100E200001C090E05E2D507143FF3CC0911102C0A3
:100E300083E001C084E0811718F4212F281B01C032
:100E400020E051110BC0F601822F30E2882319F007
:100E500031938150FBCFC20ED11C20E0992329F0A1
:100E6000D6019C93F60131966F01C6010396E2FE0E
:100E70000AC03EE4D6013C9341E411964C9311978D
:100E800012963C9306C03EE6F601308341E641836C
:100E90003283FC01322F40E2332309F442C04193F4
:100EA0003150FACF42FF44C0911102C083E001C02B
:100EB00084E0811718F4212F281B01C020E0511174
:100EC0000BC0F601822F30E2882319F03193815054
:100ED000FBCFC20ED11C20E0992329F0D6019C93B0
:100EE000F60131966F01C6010396E2FE0BC039E4AC
:100EF000D6013C933EE411963C93119736E412964A
:100F00003C9307C039E6F60130833EE6318336E68E
:100F10003283FC01322F40E2332319F041933150E8
:100F2000FBCFFC01E20FF11D10828EEF9FEFA6C0F8
:100F300021E030E0911102C020E030E016161706E3
:100F40001CF4FB01319602C0E1E0F0E02E0F3F1FE0
:100F5000BB2021F0EB2DF0E0319602C0E0E0F0E0A4
:100F60002E0F3F1FE12FF0E02E173F071CF4121B3E
:100F7000212F01C020E08E2D887159F4F601822FB7
:100F800030E2882319F031938150FBCFC20ED11C7F
:100F900020E0992329F0D6019C93F60131966F0148
:100FA00051110BC0F601822F90E3882319F0919321
:100FB0008150FBCFC20ED11C20E00F2D060F9A816D
:100FC000342F307144FF03C0913309F401501016DF
:100FD00024F4093018F008E001C001E0AB0177FF0C
:100FE00002C040E050E0FB01E41BF50BA1E0B0E0E3
:100FF000AC0FBD1FEA0FFB1F8EE2A82E4B01801A1B
:1010000091080B2D10E01195019511094F3FBFEF8D
:101010005B0721F4D601AC9211966D016417750738
:101020002CF08416950614F4818101C080E34150B0
:1010300051093196D60111967D014017510724F0D0
:10104000D6018C936701E2CF6417750739F49633A4
:1010500020F4953319F4311101C081E3F601808346
:10106000F701822F90E2882319F091938150FBCFF2
:10107000F701E20FF11D108280E090E029960FB693
:10108000F894DEBF0FBECDBFDF91CF911F910F91BE
:10109000FF90EF90DF90CF90BF90AF909F908F9098
:1010A0000895283008F027E03327DA01990F311D21
:1010B00087FD916000966105710539F432602E5FFD
:1010C0003D9330E32A95E1F708959F3F30F0803853
:1010D0007105610509F03C5F3C5F3D93913008F07C
:1010E0008068911DDF93CF931F930F93FF92EF9230
:1010F000192F987F9695E92F96959695E90FFF27DA
:10110000EA51FF4F99273327EE24FF24A701E70177
:1011100005900894079428F4360FE71EF81E491F1F
:10112000511D660F771F881F991F0694A1F7059020
:10113000079428F4E70EF81E491F561FC11D770FAC
:10114000881F991F661F0694A1F70590079428F43D
:10115000F80E491F561FC71FD11D880F991F661F04
:10116000771F0694A1F70590079420F4490F561FA6
:10117000C71FD81F990F661F771F881F0694A9F7EE
:1011800084911095177041F0D695C795579547955E
:10119000F794E7941A95C1F7ECE8F0E0689415909D
:1011A000159135916591959105907FE27395E118C0
:1011B000F10A430B560BC90BD009C0F7E10CF11E25
:1011C000431F561FC91FD01D7EF4703311F48A953A
:1011D000E6CFE894015030F0080F0AF40027021718
:1011E00008F4202F2395022F7A3328F079E37D939A
:1011F0002A95E9F710C07D932A9589F6069497956C
:101200006795379517951794E118F10A430B560B1C
:10121000C90BD00998F023957E9173957A3308F025
:1012200070E37C932013B8F77E9170617D9330F06A
:10123000839571E37D9370E32A95E1F71124EF9094
:10124000FF900F911F91CF91DF91992787FD909586
:101250000895FC010590615070400110D8F7809509
:1012600090958E0F9F1F0895FC0161507040019072
:101270000110D8F7809590958E0F9F1F08950F93BA
:101280001F93CF93DF93FB01238121FD03C08FEFD9
:101290009FEF2CC022FF16C04681578124813581E3
:1012A0004217530744F4A081B1819D012F5F3F4F46
:1012B000318320838C93268137812F5F3F4F378383
:1012C000268314C08B01EC01FB010084F185E02D25
:1012D0000995892BE1F6D80116968D919C91179767
:1012E000019617969C938E931697CE01DF91CF911E
:1012F0001F910F910895FA01AA27283051F120314A
:1013000081F1E8946F936E7F6E5F7F4F8F4F9F4F99
:10131000AF4FB1E03ED0B4E03CD0670F781F891FDB
:101320009A1FA11D680F791F8A1F911DA11D6A0FA9
:10133000711D811D911DA11D20D009F468943F915C
:101340002AE0269F11243019305D3193DEF6CF015B
:101350000895462F4770405D4193B3E00FD0C9F721
:10136000F6CF462F4F70405D4A3318F0495D31FD8E
:101370004052419302D0A9F7EACFB4E0A6959795E1
:10138000879577956795BA95C9F7009761057105B7
:1013900008959B01AC010A2E069457954795379501
:1013A0002795BA95C9F7620F731F841F951FA01D5B
:0613B0000895F894FFCF40
:1013B60001080C0406020301090901030206040CD4
:1013C600080125640025733A20252E3366202573EF
:0813D60000257320636D000087
:00000001FF
